:1000000000308A005B2A00000A108A100A11820759
:1000100028340C34013406340A108A100A1182077D
:10002000413454342B3443344D3447344C343D3410
:1000300030340D3400340A108A100A1182070C344F
:100040004E3465346E34693420346E346F34763413
:100050006134203453344D34533420347A34703482
:10006000723461347634613400340A108A100A1113
:1000700082075A34613473346C34653474346534B3
:10008000203453344D34533420346E3461342034AE
:100090006334693473346C346F3400340A108A105A
:1000A0000A1182072034203420342034373433348A
:1000B0003634203436343534353420343234353423
:1000C000303400340A108A100A1182070C3450347C
:1000D000723469346A346134743461342034533492
:1000E0004D345334203473342034743465347834CC
:1000F000743465346D3400340A108A100A11820792
:10010000413454342B3443344D34473444343D3437
:1001100031340D3400340A108A100A1182070C346D
:1001200020344F34643473347434723461346E3434
:1001300065346E3469342034763465346C346B3411
:1001400079346334683400340A108A100A11820743
:1001500020342034203420342034203420347034AF
:10016000693473346D3465346E3400340A108A1087
:100170000A11820720345A34613470346E34753475
:1001800074346F3420347A346134723469347A349C
:1001900065346E3469342034313400340A108A10E6
:1001A0000A11820720345634793470346E34753431
:1001B00074346F3420347A346134723469347A346C
:1001C00065346E3469342034313400340A108A10B6
:1001D0000A118207203420345034723465346A3472
:1001E00069342034683465347A346B34793420349B
:1001F000643465346E34213400340A148A100A11D0
:10020000820720342034203420345034723469344E
:100210006B3461347A3420346E346534623479342A
:100220006C3400340A148A100A11820720342034F6
:10023000203420342034203472346F347A346534DE
:100240007A346E3461346E3400349A30840083170B
:10025000000803193C290130F800BF30F7006400A2
:10026000F70B2F29F80B2D294A30F700F70B362909
:1002700000006400800B2B2900340708F039831636
:100280000317A10020080F392104831203138700EC
:1002900006148316061064002030F700F70B4E2971
:1002A0005129831206108316061083120034831618
:1002B00003179E08031D6229831203138610652904
:1002C00083160317831203138614831686100317ED
:1002D0009F0E1F08A000831203133D2183160317EE
:1002E0009F0E1F08A000831203133D2164004230BB
:1002F000F700F70B792900341430831603179A009E
:10030000831203132521F03083168705831286108C
:1003100083168610831206108316061003179701A2
:100320001708023C031CA42902309A00831203130D
:100330002521033083160317A000831203133D21E8
:1003400083160317970A902964000C30F700F70B07
:10035000A729AA290230A000831203133D216400BB
:100360000C30F700F70BB229B52983160317970154
:100370001708023C031CD429170883120313042016
:100380008316031798009E0118089F008312031319
:1003900057210230831603179A0083120313252175
:1003A00083160317970AB82983120313BE2A013054
:1003B000831603171B02FC3E0318F729043E831221
:1003C0000313042A831603179C01F7294030831670
:1003D00003179C00F7291430831603179C00F72994
:1003E0005430831603179C00F72983160317013036
:1003F0001A029C071C0880389D009E011D089F0062
:1004000083120313572100340A108A140A11820739
:10041000E229E629EB29F0298316031719080C3A7B
:100420008312031303191E2A063A03192E2A073AC8
:100430000319382A053A0319412A4A2A8316031751
:100440009E0101309F00831203135721023083164F
:1004500003179A008312031325215A2A01308316A9
:1004600003179A0002309B0083120313D7215A2AE4
:100470000130831603179A009B0083120313D721C0
:100480005A2A831603179E0110309F00831203130C
:1004900057215A2A8316031719081F3C031C522A96
:1004A0000730990501309E0019089F00831203133D
:1004B00057215A2A0034840183131F3083050C30DE
:1004C00083169900A6309800903083129800831606
:1004D0001F149F141F159F1107309C00FF308312BB
:1004E000A00083161F149F141F159F1183121F1045
:1004F0008316091283129412A01220088316870013
:10050000831220162008831687008312A01120086A
:100510008316870001308312940000308316940004
:100520000108C73908388100831290010030F800B3
:10053000920000308316920007309C00050864008A
:100540000230F700F70BA22AA52A1C0883120D130C
:1005500083169D010F30F70007308312810181302F
:10056000840083130008F039073880006400000815
:10057000F739F719F039770480007C296400831675
:100580000512831205129630831603179A00831200
:100590000313252183160512831205169630831640
:1005A00003179A0083120313252183160512831261
:1005B00005129630831603179A0083120313252120
:1005C00083160512831205169630831603179A00B8
:1005D000831203132521A80128080C20A80AF7007C
:1005E00077080C1EF12A99000A302802031DEC2A14
:1005F0001030840083178403840A8C1EFD2A1A0895
:1006000080000D300002031DFC2A80018C1E062B89
:100610001A088C1E092B1A081030840083178403D3
:10062000840A8C1E112B1A0880000D300002031D55
:10063000102B8001031710084F3C031D7F2B11085E
:100640004B3C031D7F2B013083169A009B008312C5
:100650000313D721A80128081B20A80AF700831636
:1006600003179900831203130C2215302802031D6F
:100670002B2B0130831603179A0002309B00831244
:100680000313D7210130831603179A0003309B0010
:1006900083120313D721A80128083520A80AF700E0
:1006A000831603179900831203130C2214302802B7
:1006B000031D4C2B0130831603179A0004309B0056
:1006C00083120313D721A80128084E20A80AF70097
:1006D000831603179900831203130C220F3028028C
:1006E000031D642B1430A800FA30831603179A00F8
:1006F000831203132521A80B742B7E2E03170313DB
:10070000A1012108363C031C8A2B8C1E852B1A085C
:10071000A10A812B8C1E8A2B1A0803179000031341
:100720008C1E902B1A080317910003138C1E962B16
:100730001A080317920003138C1E9C2B1A08031728
:10074000930003138C1EA22B1A08031794000313A3
:100750008C1EA82B1A080317950003138C1EAE2BB2
:100760001A080317960003138C1EB42B1A080317DC
:1007700097009008031DBE2B30309100303090025E
:1007800091021008093C0318C72B0730900211088A
:10079000093C0318CD2B07309102900EF0309005E4
:1007A000110890049208031DD72B3030930030308D
:1007B000920293021208093C0318E02B07309202C0
:1007C0001308093C0318E62B07309302920EF03011
:1007D0009205130892049408031DF02B3030950005
:1007E0003030940295021408093C0318F92B0730A5
:1007F00094021508093C0318FF2B07309502940E4C
:10080000F0309405150894049608031D092C303027
:1008100097003030960297021608093C0318122CF4
:10082000073096021708093C0318182C0730970266
:10083000960EF030960517089604120891001408D9
:1008400092001608930096010313A301A101210849
:10085000033C031C9C2C0310A60CA6171030210788
:100860008400831700082605A40010302107F80033
:100870000130FA000318FA0A7808A8007A08A900DB
:1008800010302107840083170008F7002308F800C0
:1008900003194E2C0310F70DF80B4A2C280884007E
:1008A00083132918831777088000A2012308083CC6
:1008B00022020318602C0310A50CA513A20A562CC3
:1008C00010302107F8000130FA000318FA0A10303E
:1008D00021078400831700082504AB0078088400F2
:1008E00083137A1883172B08800010302107F80033
:1008F0000130FA000318FA0A103021078400831728
:1009000000087F39AB007808840083137A188317B6
:100910002B0880002408A500A30A2308083C031D17
:100920009A2CA30101302107103E8400831725086B
:100930008000A601A10A272C10302107840083170C
:1009400080010130831603179A009B008312031362
:10095000D721A80128086220A80AF70083160317E8
:100960009900831203130C2215302802031DAA2CB0
:100970000930831603179A0003309B008312031378
:10098000D721103084008317003000040319DC2CB9
:10099000A9010408A8002910831B29140008831644
:1009A00003179900831203130C2228088400831371
:1009B00029188317840AC42C831605128312051282
:1009C0001430A800FA30831603179A008312031319
:1009D0002521A80BE22C8316051283120516A80107
:1009E00028087C20A80AF70077080C1EF52C99002F
:1009F0000A302802031DF02C03171008403C03188E
:100A0000072D10085A3C031C072D203090071108B1
:100A1000403C0318112D11085A3C031C112D2030A5
:100A200091071208403C03181B2D12085A3C031C66
:100A30001B2D203092071308403C0318252D130866
:100A40005A3C031C252D20309307013083169A0051
:100A50009B0083120313D721A80128088B20A80A22
:100A6000F700831603179900831203130C22143026
:100A70002802031D2D2D0130831603179A00023022
:100A80009B0083120313D721A8012808A420A80AD9
:100A9000F700831603179900831203130C220D30FD
:100AA0002802031D452D0930831603179A000430D0
:100AB0009B0083120313D72110308400831700306A
:100AC00000040319772DA9010408A8002910831B2D
:100AD00029140008831603179900831203130C22AC
:100AE00028088400831329188317840A5F2D83162E
:100AF0000512831205121430A800FA30831603176A
:100B00009A00831203132521A80B7D2D831605124D
:100B100083120516031710087A3C031D9F2D110838
:100B2000613C031D9F2D1208703C031D9F2D13086F
:100B3000313C031D9F2D01300313A700031710083C
:100B4000763C031DB32D1108793C031DB32D12080B
:100B5000703C031DB32D1308313C031DB32D02302F
:100B60000313A70003171008613C031DC72D1108CC
:100B7000683C031DC72D12086F3C031DC72D1308C9
:100B80006A3C031DC72D03300313A700031703138B
:100B90002708013A0319D32D033A0319F72D013A17
:100BA00003191B2E3B2E83168511831285110C30E1
:100BB000831603179900831203130C220130831646
:100BC00003179A0002309B0083120313D721A80158
:100BD0002808B620A80AF700831603179900831285
:100BE00003130C2213302802031DE82D732E8316E5
:100BF0008511831285150C30831603179900831213
:100C000003130C220130831603179A0002309B0055
:100C100083120313D721A8012808CE20A80AF700C1
:100C2000831603179900831203130C221330280232
:100C3000031D0C2E732E0C3083160317990083129C
:100C400003130C220130831603179A0002309B0015
:100C500083120313D721A8012808E620A80AF70069
:100C6000831603179900831203130C2212302802F3
:100C7000031D2C2E732E0C3083160317990083123C
:100C800003130C220130831603179A0002309B00D5
:100C900083120313D721A8012808FD20A80AF70012
:100CA000831603179900831203130C2210302802B5
:100CB000031D4C2E0130831603179A0003309B004E
:100CC00083120313D721A80128081221A80AF700CC
:100CD000831603179900831203130C220E30280287
:100CE000031D642E732E1430A800FA3083160317E8
:100CF0009A00831203132521A80B752EBE2A6300C8
:02400E003D3F34
:00000001FF
